:1006B80090E600E054E74410F090E601E04440F092
:1006C80090E61074A0F090E611F000000090E61299
:1006D80074A2F000000090E61374A0F000000090EF
:1006E800E61474E2F000000090E61574E0F00000F3
:1006F8000090E6917480F0000000F000000090E6A1
:1007080095F0000000F043AF01438E08758901534E
:1007180088DF43881075B2FF75B3FF75B5FFE4F540
:0907280080F590F5B043A802220F
:1003F400E5AA20E066E5AA20E56174F0F59A7400A8
:10040400F59B74F8F59D7400F59E90E690E0FE90DF
:10041400E691E07C002400F51BEC3EF51AE4F518A7
:10042400F519C3E519951BE518951A501290E67B4A
:10043400E090E67CF00519E51970E7051880E39073
:10044400E690E090E698F000000090E691E090E6F7
:1004540099F000000090E6917480F0E5AA20E2662D
:10046400E5AA20E76174F4F59A7400F59B74FCF531
:100474009D7400F59E90E694E0FE90E695E07C0085
:100484002400F51BEC3EF51AE4F518F519C3E5193B
:10049400951BE518951A501290E67BE090E67CF0E7
:1004A4000519E51970E7051880E390E694E090E6F5
:1004B4009CF000000090E695E090E69DF0000000BE
:0604C40090E6957480F043
:0104CA00220F
:02005100D322B8
:0204FE00D32207
:0205F900D3220B
:0800030090E6BAE0F51DD322DE
:1008A00090E740E51DF0E490E68AF090E68B04F0D6
:0208B000D32251
:0808DF0090E6BAE0F51CD322FB
:1008B20090E740E51CF0E490E68AF090E68B04F0C5
:0208C200D3223F
:0205FB00D32209
:0205FD00D32207
:0208E700D3221A
:10082B0090E6B9E0242F600804700A7580FF8007FA
:09083B00E4F5808002D322C322FF
:10084400C0E0C083C082D2015391EF90E65D740191
:08085400F0D082D083D0E03225
:10087400C0E0C083C0825391EF90E65D7404F0D071
:0608840082D083D0E032B7
:10088A00C0E0C083C0825391EF90E65D7402F0D05D
:06089A0082D083D0E032A1
:10077700C0E0C083C082852B27852C2885288285E9
:100787002783A37402F085232985242A852A828555
:100797002983A37407F05391EF90E65D7410F0D0AE
:0607A70082D083D0E03295
:10085C00C0E0C083C082D2035391EF90E65D740870
:08086C00F0D082D083D0E0320D
:1005BC00C0E0C083C08290E680E030E7208523272E
:1005CC00852428852882852783A37402F0852B290E
:1005DC00852C2A852A82852983A37407F05391EFF1
:0D05EC0090E65D7420F0D082D083D0E03224
:01004200328B
:0105FF0032C9
:0108E90032DC
:0108EA0032DB
:0108EB0032DA
:0108EC0032D9
:0108ED0032D8
:0108EE0032D7
:0108EF0032D6
:0108F00032D5
:0108F10032D4
:0108F20032D3
:0108F30032D2
:0108F40032D1
:0108F50032D0
:0108F60032CF
:0108F70032CE
:0108F80032CD
:0108F90032CC
:0108FA0032CB
:0108FB0032CA
:0108FC0032C9
:0108FD0032C8
:0108FE0032C7
:0108FF0032C6
:0109000032C4
:0109010032C3
:0109020032C2
:0109030032C1
:0109040032C0
:0109050032BF
:0109060032BE
:0109070032BD
:0109080032BC
:0109090032BB
:01090A0032BA
:03004300020600B2
:03005300020600A2
:100600000208440002088A000208740002085C0024
:10061000020777000205BC00020042000205FF004D
:100620000208E9000208EA000208EB000208EC00F8
:100630000208ED000208EE000208EF000208F000D8
:100640000208F1000205FF000208F2000208F300B0
:100650000208F4000208F5000208F6000208F7009C
:100660000208F8000205FF000205FF000205FF0076
:100670000208F9000208FA000208FB000208FC0068
:100680000208FD000208FE000208FF000209000047
:100690000209010002090200020903000209040024
:1006A0000209050002090600020907000209080004
:0806B0000209090002090A0019
:100500001201000200000040AD00000000000102E6
:1005100003010A06000200000040010009022E004B
:1005200001010080320904000004FF0000000705FB
:10053000020200020007050402000200070586020D
:100540000002000705880200020009022E000101D6
:100550000080320904000004FF00000007050202C9
:100560004000000705040240000007058602400025
:10057000000705880240000004030904200341002D
:10058000630071007500690072006500200044007E
:100590006500760069006300650073001403530072
:1005A000650072004D006F0064002D0035003600BC
:0C05B0000A03760031002E00300000002D
:0A08D50000010202030304040505FC
:03000B00020804E4
:10080400C0E0E52245217014758C63758ABF63903E
:10081400FF63B0FF7521017522908008E52215223F
:0708240070021521D0E03243
:10028D00E4F513F512F511F510C203C200C202C256
:10029D00011206B87E057F008E258F26752D0575FA
:1002AD002E1275230575241C752B05752C4A752F7B
:1002BD0005753078EE54C0700302038E7514007509
:1002CD0015808E168F17C374BA9FFF74059ECF24A9
:1002DD0002CF3400FEE48F0F8E0EF50DF50CF50BED
:1002ED00F50AF509F508AF0FAE0EAD0DAC0CAB0B65
:1002FD00AA0AA909A808C31208C45033E517250B8B
:10030D00F582E516350AF583E0FFE515250BF58237
:10031D00E514350AF583EFF0E50B2401F50BE43513
:10032D000AF50AE43509F509E43508F50880B785BD
:10033D00142585152674002480FF740534FFFEC333
:10034D00E52E9FF52EE52D9EF52DC3E5289FF5286D
:10035D00E5279EF527C3E52A9FF52AE5299EF52970
:10036D00C3E5249FF524E5239EF523C3E52C9FF5D6
:10037D002CE52B9EF52BC3E5309FF530E52F9EF533
:10038D002FD2E843D82090E668E04409F090E65C6F
:10039D00E04435F0D2AF90E680E020E105D20412C2
:1003AD0004CB90E680E054F7F0538EF8C2031203AD
:1003BD00F4300105120056C2013003F21200515003
:1003CD00EDC20312000E20001690E682E030E70425
:1003DD00E020E1EF90E682E030E604E020E0E41278
:0703ED0007AD1204FE80C7FA
:0B00460090E50DE030E402C322D3225D
:1000560090E6B9E0700302011514700302019224C0
:10006600FE700302021524FB700302010F147003D5
:100076000201091470030200FD1470030201032437
:100086000560030202791205F9400302028590E633
:10009600BBE024FE602714603824FD60111460273D
:1000A60024067050E52590E6B3F0E526803C120064
:1000B60046503EE52D90E6B3F0E52E802DE52790DF
:1000C600E6B3F0E5288023E52990E6B3F0E52A803B
:1000D6001990E6BAE0FF1207D9AA06A9077B01EA3A
:1000E600494B600DEE90E6B3F0EF90E6B4F00202F5
:1000F600850202740202741208B20202851208DF37
:100106000202851200030202851208A0020285126D
:1001160005FB400302028590E6B8E0247F601514D3
:10012600601924027063A200E43325E0FFA202E412
:10013600334F8041E490E740F0803F90E6BCE054C6
:100146007EFF7E00E0D394807C0040047D01800227
:100156007D00EC4EFEED4F24D5F58274083EF58306
:10016600E493FF3395E0FEEF24A1FFEE34E68F82A1
:10017600F583E0540190E740F0E4A3F090E68AF0BE
:1001860090E68B7402F00202850202741205FD40AD
:100196000302028590E6B8E024FE6016240260039E
:1001A60002028590E6BAE0B40105C20002028502A9
:1001B600027490E6BAE0705590E6BCE0547EFF7E8D
:1001C60000E0D394807C0040047D0180027D00EC39
:1001D6004EFEED4F24D5F58274083EF583E493FF79
:1001E6003395E0FEEF24A1FFEE34E68F82F583E03F
:1001F60054FEF090E6BCE05480131313541FFFE046
:10020600540F2F90E683F0E04420F08072805F1256
:1002160008E7506B90E6B8E024FE60192402704EA1
:1002260090E6BAE0B40104D200805490E6BAE064E5
:1002360002604C803990E6BCE0547EFF7E00E0D33D
:1002460094807C0040047D0180027D00EC4EFEED32
:100256004F24D5F58274083EF583E493FF3395E089
:10026600FEEF24A1FFEE34E68F82F583800D90E643
:10027600A0800812082B500790E6A0E04401F090F9
:06028600E6A0E04480F058
:01028C00224F
:030033000204FACA
:0404FA0053D8EF32B2
:1007AD0090E682E030E004E020E60B90E682E03057
:1007BD00E119E030E71590E680E04401F07F147E0A
:0C07CD000012073190E680E054FEF0229C
:1004CB0030040990E680E0440AF0800790E680E073
:1004DB004408F07FDC7E0512073190E65D74FFF077
:0F04EB0090E65FF05391EF90E680E054F7F02237
:0207D900A9076E
:1007DB00AE2FAF308F828E83A3E064037017AD0111
:1007EB0019ED7001228F828E83E07C002FFDEC3E91
:0807FB00FEAF0580DFE4FEFF04
:0108030022D2
:10000E0090E682E044C0F090E681F0438701000064
:04001E0000000022BC
:100731008E188F1990E600E054187012E519240103
:10074100FFE43518C313F518EF13F519801590E67A
:1007510000E05418FFBF100BE51925E0F519E51865
:1007610033F518E5191519AE18700215184E600504
:0607710012002280EE22BE
:100022007400F58690FDA57C05A3E582458370F9F1
:0100320022AB
:03000000020036C5
:0C003600787FE4F6D8FD75813002028D61
:1008C400EB9FF5F0EA9E42F0E99D42F0E89C45F08A
:0108D4002201
:00000001FF
